:020000040800F2
:1000000028050020D90000086D150008DD13000840
:1000100000000000000000000000000000000000E0
:10002000000000000000000000000000B7150008FC
:100030000000000000000000B5150008B915000818
:10004000EB000008EB000008EB000008EB000008E4
:10005000EB000008EB000008EB000008EB000008D4
:1000600000000000EB000008EB000008EB000008B7
:10007000EB000008EB00000800000000EB000008A7
:1000800000000000EB00000800000000000000007D
:10009000EB00000800000000EB000008EB00000887
:1000A000EB000008EB000008EB0000085D1C0008F6
:1000B000EB000008EB00000800000000000000005A
:1000C0000448854600F090F800480047311E0008BB
:1000D000C046C04628050020044880470448004721
:1000E000FEE7FEE7FEE7FEE7FEE7FEE72D16000867
:1000F000C100000830B50B46014600202022012433
:1001000009E00D46D5409D4205D31D469540491B4B
:100110002546954040191546521E002DF1DC30BD94
:10012000F0B51FB40646002082B005464024019178
:1001300000901BE0019922460F46304600F042F83D
:10014000049A059B801A994110D3104619462246FD
:1001500000F028F8361A8F4101972246012000212D
:10016000009F00F01FF838184D4100902046641E93
:100170000028DFDC019B00982946324607B0F0BD1D
:10018000D2B201E00270401C491EFBD2704700222F
:10019000F6E710B513460A4604461946FFF7F0FF86
:1001A000204610BD10B5202A04DB0146203A9140BC
:1001B000002010BD914020239C1A0346E3401943C0
:1001C000904010BD10B5202A04DB0846203AD040EC
:1001D000002110BD0B46D340D0402024A21A9140EC
:1001E0000843194610BD0000064C0125064E05E0E7
:1001F000E36807CC2B430C3C98471034B442F7D348
:10020000FFF762FF141F0008341F0008704770B525
:100210000024014620314A79022A03D00421C16317
:10022000012418E0026813680E25AB4313600268CE
:1002300013685B085B001360436C1C2213400122AF
:1002400015469D40036C5D604A7100220A71816B06
:10025000002900D08847204670BD70B5044600F0E4
:10026000CDF80546601C00D0641C00F0C7F8401BA8
:10027000A042FAD370BD0000F8B500230124A2E02B
:1002800027469F403A4070D04D68022D01D0122D74
:1002900014D1DD08AD002D1800952D6A5E07AC461F
:1002A000F50E0F26AE46AE406546B543AC460E6928
:1002B0007546AE4065462E43009D2E624D68012D69
:1002C00005D0022D03D0112D01D0122D16D1856835
:1002D0000326AC465D00AE46AE406546B543AC462F
:1002E000CE687546AE4065462E43866046680D79F9
:1002F000BE43ED06ED0F9D403543456006685F0047
:100300000325BD40AE46AE430D79B446AE07B60FE9
:10031000BE4065462E430660C6687546AE438D688E
:10032000BD403543C5604D68ED004BD5294D6E6B22
:1003300026436E639E08284DB6007519AC46AD681D
:100340009E07360F0F27B740BD4305273F07B8422A
:1003500001D1002715E0214FB84201D1012710E05B
:100360001F4FB84202D102270BE02BE01D4FB842CD
:1003700001D1032705E01C4FB84201D1052700E059
:100380000627B7402F436546AF60184D2E684F686B
:100390009643FF0300D516432E606E684F68964360
:1003A000BF0300D516436E60AE684F689643FF02E8
:1003B00000D51643AE60EE684F689643BF0200D585
:1003C0001643EE605B1C0A681546DD4000D057E717
:1003D000F8BD000000100240000001400004005081
:1003E00000080050000C0050001C005000040140A8
:1003F000002A01D08161704781627047014800681E
:10040000704700001400002070B502464032537857
:10041000202B1CD11378012B19D001231370242415
:100420005470046825689D432560046825681E0390
:10043000B5432560046825680D43256000680168A0
:1004400019430160202050700020107070BD022000
:1004500070BD70B5024640325378202B1BD1137803
:10046000012B18D0012414702423537003681D68D5
:10047000A5431D6005682B680F263602B3430902A9
:1004800019432960006801682143016020205070F1
:100490000020107070BD022070BD000070B5040017
:1004A00006D02546403568780026002802D005E0B1
:1004B000012070BD2E70204600F04AF8242068709C
:1004C000206801684908490001600F216068090639
:1004D00088432168086121688A680120C00382433B
:1004E0008A60E1680129A16808D0212292021143A3
:1004F00022689160E168022902D005E00143F7E734
:1005000001212268C902516021684A680F4B1A43D1
:100510004A602168CA688243CA60616920690843E9
:10052000A169090208432168C860216AE06908439B
:100530002168086020680168012211430160666437
:10054000202068702663AE70002070BD008000021D
:1005500010B586B0044614216846FFF718FE11490D
:10056000206888421BD1104CE16A02200143E162FD
:10057000E16A014003200591800200901220019061
:10058000012002900320039006200490694607484A
:10059000FFF772FEA06B012189050843A06306B036
:1005A00010BD000000580040001002400004005040
:1005B00002480168491C01607047000014000020D7
:1005C00010B508480024016840221143016020460C
:1005D00000F00AF8002801D0012401E000F01CF826
:1005E000204610BD0020024070B5054609487D2117
:1005F0000024C9000068FFF77DFD00F0F9FB00282A
:1006000001D0012404E000222946501E00F01AF80F
:10061000204670BD180000200448416B01221143A0
:100620004163816B020411438163704700100240F3
:10063000C106C90E012088400149086070470000CA
:1006400000E100E010B500F093FF10BDF8B50446DE
:100650000078544D800672D5524E0027403EB06B54
:10066000C00004D4B06BA9050843B06301274E480D
:100670000168C90511D40168821511430160FFF7B3
:10068000BDFE009005E0FFF7B9FE0099401A64280E
:1006900037D845480068C005F5D5326803210905FB
:1006A00060680A400140914208D08103890F032904
:1006B00004D13168890301D50120F8BD2A690321DD
:1006C00009040A4022D0084090421FD020788006BA
:1006D0001CD528692A6988430121C9040A432A6173
:1006E0002A698A432A612861C0050FD5FFF786FE73
:1006F000009008E0FFF782FE0099411A2B488142E2
:1007000001D90320F8BD28698005F3D56168880305
:10071000800F032805D132680005824301400A4357
:10072000326028690322616812041140084328617D
:10073000002F04D0B16B012000078143B163207802
:10074000C00705D0E868A168800880000843E86019
:100750002078800705D5E8680C218843E1680843C4
:10076000E8602078400706D5E868032189028843BD
:1007700021690843E8602078000706D5E86803216E
:100780000903884361690843E8602078000606D5BC
:10079000E868032189048843A1690843E8600020D0
:1007A000F8BD0000401002400070004088130000B7
:1007B000F8B50E4605007DD053480068C007C00F4D
:1007C000B0420AD2504801684908490031430160EB
:1007D0000068C007C00FB04271D128784B4C800729
:1007E00005D5E068F0218843A9680843E0602878CF
:1007F000C00752D06868022817D0032818D0216893
:10080000012818D08905002959DAE168890889008A
:100810000143E160FFF7F2FD69680746022912D043
:1008200003291CD0012926D033E021688903EAE797
:1008300021688901E7E74907E5E7FFF7DFFDC11B0D
:100840003348814223D8E0680007800F0228F4D1A2
:1008500023E0FFF7D3FDC11B2D48814217D8E06884
:100860000007800F0328F4D117E0FFF7C7FDC11B75
:10087000274881420BD8E0680007800F0128F4D197
:100880000BE0FFF7BBFDC11B2148814201D90320CA
:10089000F8BDE0680007800FF3D11B480168C90765
:1008A000C90FB1420DD901684908490031430160BF
:1008B000006800E003E0C007C00FB04201D0012093
:1008C000F8BD2878400706D5E0680721090288436B
:1008D000E9680843E0602878000707D5E068072149
:1008E000C90288432969C9000843E06000F036F86E
:1008F000E168084A0906090F515CC84006490860CA
:100900000020FFF771FEF8BD0020024000100240F9
:1009100088130000F01E0008180000200448054954
:100920000068C968044A4905490F515CC8407047CE
:100930001800002000100240091F00080448054963
:100940000068C968044A8904490F515CC84070476F
:100950001800002000100240091F000810B5184AB6
:10096000D1680C20084004280BD0082810D00C288F
:1009700010D050680004410F0120C003491C88407A
:1009800010BD1068C00601D50E4810BD0E4810BD40
:100990000E4810BD88020E4B000F185C0902D36888
:1009A000890F491CDB0301D5084A05E01268D2060D
:1009B00001D5044A00E0044A5043FFF79BFB10BDF9
:1009C0000010024000093D000024F40000127A00EB
:1009D000001F0008FEB505007ED0FE4CE7680C2025
:1009E000E66807400120000406402878C00747D089
:1009F000082F05D00C2F0AD101200004864206D111
:100A0000206880033CD568680028E5D038E00120E4
:100A100069680004814203D121680143216011E02B
:100A2000052301221B0492049942216802D111433B
:100A30002160F1E781432160216801400091206835
:100A400090432060686800280DD0FFF7D7FC009025
:100A500005E0FFF7D3FC0099401A64287AD8206893
:100A60008003F6D50CE0FFF7C9FC009005E0FFF726
:100A7000C5FC0099401A6428F0D820688003F6D499
:100A80002878800755D50923E868042F0DD00C2F4E
:100A900001D1002E09D000283BD0216899430143A1
:100AA0002160FFF7ABFC064627E02168490701D526
:100AB000002891D061681F22120291432A69120214
:100AC000114361602168994301432160FFF746FFAC
:100AD000E16809060A0F00E079E1BF49895CC84076
:100AE000BE4908600020FFF77FFD002872D120E09A
:100AF000FFF784FC801B0228B0D820684007F7D598
:100B000060681F210902884329690902084360605F
:100B10000FE02068400840002060FFF76FFC0646A9
:100B200004E0FFF76BFC801B022897D82068400781
:100B3000F7D42878C0065FD5002F0CD0A86900280C
:100B400049D02068FF21013108432060FFF756FC9F
:100B500006462DE0C0E02068800502D5A86900287F
:100B6000A7D06068072149038843296A0843606069
:100B70006068297F0002000A090608436060286A4D
:100B8000410B0120C003491C8840E16809060A0F97
:100B90009149895CC840914908600020FFF724FD15
:100BA000002817D128E0FFF729FC801B0228A3D8D2
:100BB00020688005F7D56068072149038843296AC2
:100BC000084360606068297F0002000A0906084344
:100BD000606011E0E1E02168FF2001308143216085
:100BE000FFF70CFC064604E0FFF708FC801B022818
:100BF00072D820688005F7D42878794E000724D56C
:100C000068690028306910D0012108433061FFF77E
:100C1000F5FB009005E0FFF7F1FB0099401A022870
:100C20005AD830698007F6D50FE04008400030619F
:100C3000FFF7E4FB009005E0FFF7E0FB0099401AA6
:100C4000022849D830698007F6D42878400765D54E
:100C500000200290A06BC00006D4A06B0121090700
:100C60000843A063012002905E480168C90511D4C1
:100C70000168821511430160FFF7C0FB009005E099
:100C8000FFF7BCFB0099401A642825D85548006836
:100C9000C005F5D5FF20AA680130824203D1316931
:100CA0000143316111E001218902002A07D00523A7
:100CB0001B029A4203D132690A433261EFE732697B
:100CC00082433261306988433061A86800280FD0C0
:100CD000FFF794FB009007E05EE0FFF78FFB0099C1
:100CE000411A4148814257D830698005F5D50DE059
:100CF000FFF784FB009006E0FFF780FB0099411AA4
:100D00003948814248D830698005F5D402980028D6
:100D100004D0A06B012109078843A063686A0028FA
:100D200064D00C2F3ED0012636060228206805D05C
:100D3000B0432060FFF762FB05462FE0B043206020
:100D4000FFF75CFB074604E0FFF758FBC01B0228D7
:100D500022D820688001F7D4E96AA86AE2680843CB
:100D6000296BFD231B049A4311430843E06020686C
:100D700030432060FFF742FB054604E0FFF73EFBEF
:100D8000401B022808D820688001F7D52EE0FFF725
:100D900035FB401B022801D90320FEBD20688001DD
:100DA000F5D423E00128F8D0E06801210904AA6AFB
:100DB000014091420BD10F218904EA6A014091421E
:100DC00005D1032189050840296B88420ED00120F6
:100DD000FEBD000000100240F01E000818000020B8
:100DE0004010024000700040881300000020EFE730
:100DF000094910B5401E884201D9012010BD074C99
:100E000060610321081F00F0B3FB0020A0610720F0
:100E10002061002010BD0000FFFFFF0000E000E0A7
:100E2000F0B502462032137E012B15D0012717762C
:100E30000223537605686C68AB687026B4430E686D
:100E4000496826438024A34319436E60006881608B
:100E5000577600201076F0BD0220F0BD10B586B0A8
:100E6000044614216846FFF792F90D49206888422C
:100E700013D10C48C26A02210A43C262C06A0191BE
:100E8000084005903020009000200290039004203C
:100E9000049069460448FFF7EFF906B010BD000062
:100EA000001401400010024000040050F8B506464E
:100EB00004462036307E0D4601280DD001203076C4
:100EC000022070760427002A08D0042A16D0082AA7
:100ED0002AD00C2A4DD137E00220F8BD206800F05E
:100EE00008FC2068816908221143816120688169BA
:100EF000B943816120688169EA6812E0206800F0E6
:100F000010FC206882690121C9020A4382612068BD
:100F10008169012292029143816120688169EA68B6
:100F200012021143816124E0206800F013FC206864
:100F3000C26908210A43C2612068C169B943C1611D
:100F40002068C169EA6812E0206800F01EFC206891
:100F5000C1690122D2021143C1612068C269012125
:100F600089028A43C2612068C169EA68120211439A
:100F7000C1610120707600203076F8BD70B50400A4
:100F800005D025462035687E002802D006E00120E5
:100F900070BD00202876204600F00AF8022068760E
:100FA000211D206800F06CFB01206876002070BDD8
:100FB00000680449884204D10348416B2022114350
:100FC00041637047001401400010024010B5044610
:100FD0000068012200F080FB206881684907490F02
:100FE000062903D00168012211430160002010BDD1
:100FF00070477047F8B502680446D0691168936875
:1010000005072D0F5BD0DD07ED0FFF2621360E40C3
:101010002E4367D0C60706D0CE0504D5012616623A
:10102000E26F3243E267870702220426002F06DAC6
:10103000DF0704D027683A62E76F3743E76747075F
:1010400006D5DB0704D023681E62E36F1343E36712
:10105000020709D520220A402A4305D02368082226
:101060001A62E36F1343E367E26F002A2FD0800612
:1010700006D5880604D5216E002901D02046884770
:10108000E06F21688968490601D4000724D520460D
:1010900000F036FC20688168490619D58168402235
:1010A00091438160E06E002812D020498163E06E98
:1010B000FFF7ADF800280AD0E06E816B06E08506E8
:1010C00010D58D060ED5216E1CE020468847F8BD50
:1010D0002046FFF78EFFF8BD2046FFF78AFF00206D
:1010E000E067F8BDC50208D55B0206D50120000502
:1010F00010622046FFF77CFFF8BD030605D50B06FE
:1011000003D5616E0029E0D1F8BD4006FCD5480644
:10111000FAD51368204640218B4313602021616774
:101120000021616600F059F9F8BD0000ED180008D3
:1011300010B5040003D0606F002802D007E0012042
:1011400010BD002170200155204600F027F8242012
:10115000606720680168490849000160204600F086
:1011600037FC0128ECD0606A002802D0204600F04D
:1011700027FB206841680922D20291434160206820
:1011800081682A229143816020680168012211430D
:101190000160204600F07AFB10BD000010B586B05B
:1011A000044614216846FEF7F2FF1549206888427C
:1011B00024D11448416B0122920311434163C16A57
:1011C00001221143C162C06A6946104005900320A4
:1011D0004002009002200190002002900320039022
:1011E0000420049005200007FFF746F8002211466E
:1011F0001B20FFF727FA1B20FFF71AFA06B010BDD5
:101200000038014000100240F0B5836F202B54D10C
:1012100000290AD0002A08D08568DC01A54206D141
:101220000369002B03D1CB0701D00120F0BD034699
:1012300060331E7C012E40D001261E74416501469C
:1012400040310A834A830022FF260266A54204D168
:101250000569002D13D11A4D0AE07F27002D09D012
:1012600001263607B5420CD10569002D05D03F2572
:101270008D8307E00569002D01D08F8302E08E8306
:1012800000E08A83C2672221816701688D68012698
:1012900035438D608168A14202D1016900290AD0DD
:1012A000084901661A7400680168FF22213211435F
:1012B00001600020F0BD0449F3E70220F0BD00000A
:1012C000FF010000791900082119000810B50C4829
:1012D0000178FF2902D181790D2907D008493223ED
:1012E0000522491F074800F011F810BD044A417853
:1012F0000D3A51608078106003A000F0B7FC10BD7B
:101300000D000020A800002025640000FFB5044661
:10131000406F83B017460D4620285CD1002D0AD0BF
:10132000002F08D0A168C001814207D120690028A0
:1013300004D1E80702D0012007B0F0BD204660309C
:101340000290007C012846D00298012101740020FF
:10135000E06721206067FFF751F82646403601908C
:10136000378277820120A1680003814202D120697F
:10137000002802D02F46002511E000270FE00022B0
:101380008021204600F038FC002815D1002F15D010
:101390002168387888627F1C708A401E7082708A4B
:1013A000019B002806980090E9D1002240212046A8
:1013B00000F022FC002808D00320BDE7288821681F
:1013C000C005C00D8862AD1CE6E720206067029969
:1013D00000200874B0E70220AEE77047FEE7000087
:1013E000F0B587B014216846FEF7D1FE1848C26AEE
:1013F00002210A43C262C26A0A400592C16A0125FB
:101400002943C162C06A032428400526E402360746
:101410000590002221463046FEF7EAFF0D4F0022DC
:1014200040213846FEF7E4FF009400240195029421
:10143000694630460394FEF71FFF40200090029457
:101440006946019503943846FEF716FF07B0F0BDD4
:10145000001002400004005010B51348114901600B
:101460001249416000218160016141618161012275
:10147000C161C2600162FFF711F8002801D0FEF7D8
:10148000C5FE00210848FEF7BFFF002801D0FEF787
:10149000BDFE00210448FEF7DCFF002801D0FEF766
:1014A000B5FE10BD005800402000002009050000D6
:1014B00010B586B0002405941C491D48049400947E
:1014C00001940294039412C0046084606321C46098
:1014D00041600838FFF752FD002801D0FEF796FE64
:1014E000049404A912480594FFF79AFC002801D03F
:1014F000FEF78CFE60200090019402940022694661
:1015000003940B48FFF7D2FC002801D0FEF77EFEC3
:10151000042269460648FFF7C9FC002801D0FEF7FF
:1015200075FE0348FFF79AFC06B010BD0014014099
:101530006C00002010B50C480A490160E121490205
:10154000416000218160C16001618161C1610C2243
:10155000016242614162FFF7EBFD002801D0FEF716
:1015600055FE10BD00380140A80000207047000063
:101570008307FF22DB0E9A408907090E9940002855
:101580000BDA0007000F0838830808489B0018187A
:10159000C36993430B43C3617047830804489B00AE
:1015A0001B181868904308431860704700ED00E06E
:1015B00000E400E07047704710B5FEF7F9FF10BD7A
:1015C00030B599B034216846FEF7E1FD14210DA82D
:1015D000FEF7DDFD1C2112A8FEF7D9FD12480168B7
:1015E0000322D2029143C2148918016002200090A4
:1015F0000024102009940125049003956846FFF704
:10160000E9F90F200D90A0200F900E951094002165
:1016100011940DA8FFF7CCF812A812951494FFF7B7
:1016200015F819B030BD0000007000401048016886
:10163000821511430160C1680E4A1140C160016802
:101640000D4A1140016081684908490081600168C4
:101650000122920491430160C168FD22120491436A
:10166000C160002101610549C00388607047000026
:10167000001002400C40FF88F6FFF6FE00ED00E08F
:1016800070B5026801239B07114C124D984203D09C
:10169000A04201D0A84203D17026B2434E68324323
:1016A000984203D0A04201D0A84204D103231B02D8
:1016B0009A43CB681A4380239A430B691A4302600A
:1016C0008A68C262096881620121416170BD0000BF
:1016D000000801400014014010B5CB06DB0E0121CB
:1016E000046A99408C430462016A9A401143016282
:1016F00010BD30B5026A520852000262026A4568A3
:1017000083697024A3439C080B68A400234302242C
:10171000A2438C6845601443836149684163046255
:1017200030BD30B5026A10239A430262036A4568ED
:10173000826973242402A2430C68240214432022E9
:1017400093438A68456012011A4384614968816342
:10175000026230BD30B5026AFF2301339A43026250
:10176000026A4568C3697024A3439C080B68A400FF
:10177000234301246402A2438C684560240214437D
:10178000C3614968C163046230BD30B5026A012398
:101790001B039A430262036A4568C26973242402E8
:1017A000A2430C68240214430122520393438A6823
:1017B000456012031A43C46149680164026230BD86
:1017C00010B5818CC90707D001684A6801235B0402
:1017D0009A43836A1A434A60818C890707D5016856
:1017E0004A6801231B049A43C36A1A434A60818CE6
:1017F000490707D501684A6801239B049A43036B94
:101800001A434A60818C090707D501684A68012399
:10181000DB039A43436B1A434A60818CC90607D5A0
:101820000268916801231B039943836B19439160FC
:10183000818C890607D501688A6801235B039A4376
:10184000C36B1A438A60818C490612D503685A68B3
:1018500001210905046C8A4322435A60026C8A42C2
:1018600007D10268516803235B059943436C194310
:101870005160818C090607D501684A680123DB04A1
:10188000806C9A4302434A6010BD0000F8B5002600
:101890000446C667FEF7B2FD054620680068124F91
:1018A000000709D501212B46002249052046009753
:1018B00000F0A2F900280DD12068006840070BD580
:1018C00001212B46002289052046009700F094F95B
:1018D000002801D00320F8BD20206067A067603495
:1018E00026740020F8BD0000FFFFFF0110B5806ADC
:1018F0000022014640314A834A82FFF77AFB10BD3D
:1019000001680A68FF2321339A430A6001688A68E4
:10191000520852008A6020218167002101667047C9
:1019200010B5014640318B8B846F0268222C04D0A5
:10193000906908210843906110BD526A446D1A40B5
:101940002280426D921C42654A8B521E4A83498B0B
:101950000029F1D101680A68FF2321339A430A6004
:1019600001688A68520852008A602021816700213C
:101970000166FFF7ABFC10BD10B5014640318B8B03
:10198000846F0268222C04D090690821084390617A
:1019900010BD526A1A40436D1A70426D521C426566
:1019A0004A8B521E4A83498B0029F1D101680A688B
:1019B000FF2321339A430A6001688A685208520063
:1019C0008A602021816700210166FFF77FFC10BD3E
:1019D000F8B504462669A268E769324366691020B3
:1019E00000253E432368324378491E68784F3E40C5
:1019F00016431E6023685A6803263603B243E6681E
:101A000032435A602368A2698B4201D0266A32436E
:101A10009E680B273F02BE4316439E606D4E2368AF
:101A20006D4AB3420CD1D2689207920F06D0012AB8
:101A300038D0022A34D0032A20D11EE001201DE034
:101A4000664EB3420AD1D2680C26324026D0042A10
:101A500028D0082A24D00C2A10D10EE08B420DD1B8
:101A6000D66803229202164018D001229202B61ABA
:101A700018D0B61A14D0964200D10820564A012632
:101A8000403A574FF6038B4236D100280CD002283B
:101A90000DD0042812D008281FD11CE00020EDE74B
:101AA0000220EBE70420E9E7FEF738FF08E01068C2
:101AB000C00601D5384605E04A4803E0FEF74EFF70
:101AC000002873D0626851005118814205D8110373
:101AD000814202D303E03046F4E7012566E0010EBF
:101AE00006025008002330185941FEF719FB032164
:101AF0000902411A3C4A55E0E169B14232D1030082
:101B000000F0C4F809070A0D06250606062B060094
:101B1000E3E7FEF703FF1CE0FEF710FF19E0106893
:101B20006168C00602D54808304A01E0304A4808DA
:101B30008018FEF7DFFA80B201462E4A1039914232
:101B4000CBD8511C01400007400F08432CE0FEF7A2
:101B500005FF616840004A08EAE761680122480819
:101B60001204E5E7030000F091F809070A0D0626C4
:101B70000606062C0600B0E7FEF7D0FE1DE0FEF7D5
:101B8000DDFE1AE010686168C00602D54808C01979
:101B900002E014484A081018FEF7ACFA80B2014679
:101BA000144A1039914298D82168C86000202066F4
:101BB00060662846F8BDFEF7D1FE61684A088018C5
:101BC000EAE7616848088019E6E70000004800403D
:101BD000F369FFEF0038014040100240004400402C
:101BE00000093D000024F400FFFC0F0000127A0001
:101BF0000048E801EFFF0000FFB581B017460E4630
:101C000004460A9D09E0681C07D0FEF7F7FB04991B
:101C1000401AA8420CD8002D0AD02068C16930466D
:101C2000884318D00020B842EDD0002005B0F0BDA8
:101C300020680168FF22A132914301602068816819
:101C400049084900816020206067A0670020603457
:101C500020740320EAE70120E5E7000010B5024800
:101C6000FFF7C8F910BD0000A80000200FB410B5A0
:101C700003A9044B044A029800F024F810BC08BCE5
:101C800004B01847151E00081C00002030B474462C
:101C9000641E2578641CAB4200D21D46635D5B0068
:101CA000E31830BC184702E008C8121F08C1002A18
:101CB000FAD170477047002001E001C1121F002ACD
:101CC000FBD17047FFB58DB00446002506E02528FE
:101CD0000AD0109A0F999047641C6D1C2078002838
:101CE000F5D1284611B0F0BD00270121484A0097E0
:101CF00000E00743641C23780846203B98401042CC
:101D0000F7D120782E2817D1042007436078641C6F
:101D10002A280CD10E98641C02C800910E900BE08A
:101D200000990A22514330394018641C00902078F1
:101D3000014630390929F3D920780028D1D0642808
:101D400008D0692806D075281ED0109A0F999047A0
:101D50006D1C5BE00A200E99019001C90E910028CC
:101D600002DA40422D2102E0390504D52B216A46D2
:101D70001172012103E0F90704D02021F7E70BAE2F
:101D80000B910DE00021FAE70A200E99019001C99C
:101D90000E91F7E70199FEF7ADF93031761E3170FB
:101DA0000028F7D103A8801B20300190780701D5C7
:101DB000009801E0012000900199884201DD401A5D
:101DC00000E000200027009006E002A8109AC05D05
:101DD0000F9990476D1C7F1C0B988742F5DB04E040
:101DE000109A30200F9990476D1C0099481E009062
:101DF0000029F5DC05E03078109A761C0F999047A1
:101E00006D1C0199481E01900029F4DC641C65E7F3
:101E10000928010001B5044B012269460348FFF778
:101E200075FA009808BD0000FFFF0000A800002020
:101E3000FEF7C6FBFFF7C4FBFFF7D2FAFFF70CFB78
:101E4000FFF778FBFFF734FB00211248FFF7BEF8DD
:101E500004211048FFF7BAF80F4C0F4907220D3143
:101E60000E48FFF7D1F96420FEF7F7F92068002843
:101E700007D0002000F014F8A08880B200F024F809
:101E8000EBE7002000F020F8A08880B200F008F80E
:101E9000E3E700006C00002000000020A800002004
:101EA0001FB501900020602100910290024603902E
:101EB00069460448FEF7FAFF00210248FFF786F85A
:101EC0001FBD00006C0000201FB5019000206021A4
:101ED000009102900390042269460448FEF7E6FF51
:101EE00004210248FFF772F81FBD00006C000020BB
:101EF00000000000000000000102030406070809BA
:101F0000030406080C101820300000000001020332
:101F100004000000341F0008000000202000000022
:101F2000A61C0008541F000820000020080500001F
:101F3000B61C00080000000000000000FF010203C2
:101F40000D00000000000000000000000000200064
:041F5000000000008D
:04000005080000C12E
:00000001FF
